:10000000000000308A006628A7002008840021092B
:10001000841780058413A70803192C28F030A90041
:1000200026088038A800F030A9030319A900031995
:10003000A70303192C281C283020030122182108AB
:10004000A61F2108A60803190301A80F2928800666
:1000500010282A2800001328210884178004622809
:10006000230822040319A20A8030221AA3062219A7
:10007000A306A218A306230DA20DA30D2208622831
:10008000A701A600FF30A607031CA707031C6228D0
:100090000330A500DF304E204228A501E83EA40031
:1000A000A509FC30031C5728A40703185428A407EB
:1000B0000000A50F542824185D28A41C6128000006
:1000C0006128080083138312031308008301831639
:1000D00085018312850183168601831286018316AA
:1000E0008701831287010530A0001030A100323053
:1000F000A6003C308A0104204630A60014308A0154
:1001000004205530A60078308A0104205330A60020
:1001100028308A0104204630A60014308A010420C9
:100120003230A60014308A0104204630A600143074
:100130008A0104205A30A60078308A0104205A30FF
:10014000A60014308A0104206230A600A0308A0183
:1001500004200730A700D0308A0141208030AA0057
:100160000530A0001030A1002A08A60002308A0144
:1001700004200130AA078A110A12031CB028073094
:10018000A700D0308A0141200530A0001030A10026
:100190002B30A60050308A0104203F30A6001430D6
:1001A0008A0104204D30A60014308A010420473013
:1001B000A60050308A0104203330A60014308A0192
:1001C00004205A30A60014308A0104205530A600BD
:1001D0008C308A0104204D30A60014308A0104209E
:1001E0005030A60014308A0104205530A600143087
:1001F0008A0104205A30A60014308A0104205030AD
:10020000A60014308A0104205530A6003C308A0133
:1002100004205A30A6003C308A0104205C30A6003D
:100220003C308A0104205730A6003C308A0104206B
:100230006030A60046308A010420A6010A308A01F7
:1002400004206030A6000A308A010420A6010A308A
:100250008A0104206030A6000A308A010420A60129
:100260000A308A0104206030A6001E308A01042072
:10027000A6010A308A0104205C30A6001E308A01E3
:100280000420A6010A308A0104205730A6001E303F
:100290008A010420A6010A308A0104206030A600E9
:1002A00028308A010420A60114308A0104203F303E
:1002B000A6000A308A010420A6010A308A0104201F
:1002C0003F30A6000A308A010420A6010A308A01C4
:1002D00004203F30A6000A308A010420A6010A301B
:1002E0008A0104203F30A60014308A010420173010
:1002F000A70070308A0141208A01732863008A01B7
:060300007E298A0181291B
:02400E00323F3F
:00000001FF
